:100000000C9434000C9451000C9451000C94510049
:100010000C9451000C9451000C9451000C9451001C
:100020000C9451000C9451000C9451000C9451000C
:100030000C9451000C9451000C9451000C945100FC
:100040000C9451000C9451000C94CA000C94F100D3
:100050000C9418010C9451000C9451000C94510014
:100060000C9451000C94510011241FBECFEFD8E026
:10007000DEBFCDBF11E0A0E0B1E0ECEDF3E002C0E7
:1000800005900D92AA32B107D9F721E0AAE2B1E0BA
:1000900001C01D92A039B207E1F70E94A9010C949A
:1000A000EC010C940000259A2D98089595B180E2FA
:1000B000892785B908952D9A08952D980895089552
:1000C0008091C6000895E1ECF0E08081806180833A
:1000D0000895E1ECF0E08081886080830895E1EC90
:1000E000F0E090819B7F9083E2ECF0E09081997F3B
:1000F000908390818370880F982B90830895DC0102
:10010000CB01880F991FAA1FBB1F880F991FAA1F19
:10011000BB1F9C01AD01220F331F441F551F220F2F
:10012000331F441F551F60E074E284EF90E00E948B
:10013000C1018FEF820F8093C400DA01C9010197DA
:10014000A109B109892F9A2FAB2FBB278093C50036
:1001500008959093050180930401E1ECF0E0808123
:10016000806880830895E0ECF0E0908195FFFDCFFA
:100170008093C6000895CF93DF93EC018881882394
:1001800031F021960E94B30089918111FBCFDF915C
:10019000CF9108951F920F920FB60F9211242F93B3
:1001A0003F934F935F936F937F938F939F93AF93FF
:1001B000BF93EF93FF93E0910401F091050109953E
:1001C000FF91EF91BF91AF919F918F917F916F912F
:1001D0005F914F913F912F910F900FBE0F901F9005
:1001E00018951F920F920FB60F9211242F933F93E1
:1001F0004F935F936F937F938F939F93AF93BF932F
:10020000EF93FF93E0910201F09103010995FF91B3
:10021000EF91BF91AF919F918F917F916F915F917E
:100220004F913F912F910F900FBE0F901F901895F7
:100230001F920F920FB60F9211242F933F934F935B
:100240005F936F937F938F939F93AF93BF93EF933E
:10025000FF93E0910001F09101010995FF91EF9169
:10026000BF91AF919F918F917F916F915F914F91CE
:100270003F912F910F900FBE0F901F9018950E94E5
:10028000600090912A01911127C08D3051F4E091C6
:100290002B01F0E0E45DFE4F108281E080932A01A3
:1002A00008958830A9F4E0912B01EE2331F0E1505C
:1002B000E0932B010E94B300089591E09E0F90936C
:1002C0002B01F0E0E45DFE4F80830E94B3000895AF
:1002D000E0912B01E33688F30895EF92FF920F939C
:1002E0001F93CF93DF9380912A01882359F106E071
:1002F00011E0C0E0D0E06CE271E0F8018081918112
:100300000E94E301892B81F4FE01EE0FFF1FEE0F27
:10031000FF1FEA5FFE4F0280F381E02D09951092E6
:100320002B0110922A010EC021960C5F1F4FC33083
:10033000D10509F782E191E00E94BB0010922B01E8
:1003400010922A01DF91CF911F910F91FF90EF90B2
:1003500008950E945300F8940E9463000E9469006F
:1003600083E00E946F0060E875E280E090E00E9408
:100370007F008FE391E00E94A90078940E946D01B4
:10038000FDCFA1E21A2EAA1BBB1BFD010DC0AA1FA7
:10039000BB1FEE1FFF1FA217B307E407F50720F0EE
:1003A000A21BB30BE40BF50B661F771F881F991F69
:1003B0001A9469F760957095809590959B01AC01B2
:1003C000BD01CF010895FB01DC018D9101908019E1
:0C03D0000110D9F3990B0895F894FFCFA9
:1003DC005F005F005F0018015B001E015D002401DF
:1003EC0056006E6D660A0D006C65642031006C65FC
:0A03FC00642030006C65642074007A
:00000001FF
